:020000040800F2
:1000000000040220010200080302000803020008A5
:1000100003020008030200080302000803020008AC
:10002000030200080302000803020008C5260008B6
:10003000030200080302000803020008030200088C
:10004000030200080302000803020008030200087C
:100050000302000803020008DD380008093900081F
:1000600035390008613900088D390008030200089D
:10007000030200080302000803020008030200084C
:10008000030200080302000803020008030200083C
:10009000030200080302000803020008B93900083F
:1000A000030200080302000803020008030200081C
:1000B00001370008030200080302000803020008D9
:1000C00003020008030200080302000803020008FC
:1000D00003020008030200080302000803020008EC
:1000E000213A000803020008030200080302000886
:1000F00003020008030200080302000803020008CC
:1001000003020008030200080302000803020008BB
:1001100003020008030200080302000803020008AB
:10012000030200080302000803020008030200089B
:10013000030200080302000803020008030200088B
:10014000030200080302000803020008312E000821
:10015000030200080302000803020008030200086B
:10016000030200080302000803020008030200085B
:10017000030200080302000803020008030200084B
:100180000302000803020008BD0F00080302000874
:10019000030200080302000803020008030200082B
:1001A000030200080302000803020008030200081B
:1001B000030200080302000803020008030200080B
:1001C00003020008030200080302000803020008FB
:1001D00003020008030200080302000803020008EB
:1001E00003020008030200080302000803020008DB
:1001F00003020008030200080302000803020008CB
:1002000002E000F000F8FEE772B6394880F3088893
:10021000384880F3098838484EF60851CEF200017C
:10022000086040F20000CCF200004EF63471CEF2CD
:1002300000010860BFF34F8FBFF36F8F40F20000E3
:10024000C0F2F0004EF68851CEF200010860BFF314
:100250004F8FBFF36F8F4FF00000E1EE100A4EF6A4
:100260003C71CEF200010860062080F31488BFF3D1
:100270006F8F02F065FA03F0CBF94FF055301F494C
:100280001B4A91423CBF41F8040BFAE71C49194A4A
:1002900091423CBF41F8040BFAE71A491A4A1B4B3A
:1002A0009A423EBF51F8040B42F8040BF8E70020D5
:1002B0001749184A91423CBF41F8040BFAE702F093
:1002C00083FA03F00FFA144C144DAC4203DA54F8DD
:1002D000041B8847F9E700F03FF8114C114DAC4280
:1002E00003DA54F8041B8847F9E702F06BBA000000
:1002F0000004022000240220000000080000022068
:1003000000040220B03E00080024022050240220F5
:1003100050240220D8380220000200080002000801
:1003200000020008000200082DE9F04F2DED108AB0
:10033000C1F80CD0D0F80CD0BDEC108ABDE8F08F1D
:10034000002383F311882846A047002001F048FECF
:1003500001F0F8FD00DFFEE770B5214C6FF070038F
:10036000002523706FF07F061E236570A570E57071
:1003700025716571A571E57125726672A372E572CA
:1003800000F03CFD20B10E2325726672A372E57267
:1003900002F070F9044602F08FF90546D8B9114B06
:1003A0009C421AD001339C4218BF054641F2883462
:1003B00004BF01250024002002F066F90DB100F011
:1003C000B7F800F08DFD00F06BFC204600F050F90E
:1003D00000F0AEF8F9E70024EDE70446EBE700BFD4
:1003E00050240220010007B008B500F0D7FBA0F1AF
:1003F00020035842584108BD07B5054B02211B8810
:10040000ADF8043001A800F035FC03B05DF804FB42
:10041000203B0008064991F8243033B1002308221C
:10042000086A81F8243000F05FBC0120704700BFEB
:10043000702402202DE9F84F234C94F8243005460F
:10044000884617468BBB2E46DFF87C90002F38D0AD
:1004500094F824A0BAF1000F05D12022FF214846CC
:10046000266200F02BFDCAF10805BD4228BF3D46BB
:100470005FFA85FBAD0041462A4604EB8A0000F096
:10048000F3FC94F82430A7EB0B079B445FFA8BFB3B
:10049000BBF1080F2E44A844FFB284F824B0D5D194
:1004A000FFF7B8FF0028D1D108E0266A06EB8306E3
:1004B000B042C9D0FFF7AEFF0028C4D10020BDE88C
:1004C000F88F0120BDE8F88F7024022010B520239A
:1004D00083F311881248C3680BB101F007FE0023B3
:1004E000104A0F484FF47A7101F0C4FD002383F3E2
:1004F00011880D4C236813B12368013B23606368A6
:1005000013B16368013B6360084B1B7833B96368C0
:1005100023B9022000F09EFC3223636010BD00BFAF
:100520005C240220CD040008A02902209824022087
:100530002DE9F041444B454953F8042F013201D1D4
:10054000BDE8F0818B42F7D1414C424B22689A4280
:1005500078D9414B9B6803F1006303F5C0339A429D
:1005600070D2002000F0B8FB3C4B0220187000F065
:1005700067FC3B4B1A6C00221A64196E1A66196EDE
:10058000596C5A64596E5A66596E596941F0800126
:100590005961596921F0800159615969196941F01E
:1005A00000511961196921F0005119611B6972B676
:1005B0002C492D4B0B601D682468BFF34F8FBFF390
:1005C0006F8F2A4BC3F88420BFF34F8F5A6922F4F0
:1005D00080325A61BFF34F8FD3F88020C2F3C9062F
:1005E000C2F34E325201B70743F6E07E02EA0E082C
:1005F00038463146013948EA000CB1F1FF3FC3F8F3
:1006000074C200F14040F5D1203A12F1200FEDD133
:10061000BFF34F8FBFF36F8FBFF34F8FBFF36F8F5A
:100620005A6922F400325A610022C3F85022BFF303
:100630004F8FBFF36F8F202383F31188AD4685F36F
:1006400008882047BDE8F081FC7F01081C80010874
:1006500004800108FF7F0108502402209824022012
:100660000038024008ED00E00080010800ED00E0E5
:100670002DE9F04FB04C97B020228146FF210EA803
:10068000A66800F01BFCAD4A1378A346A3B9AC489A
:100690000121C3601170202383F31188C3680BB15B
:1006A00001F024FD0023A74AA5484FF47A7101F018
:1006B000E1FC002383F31188B9F1000F02D0A24BB3
:1006C000C3F80090A14BA04A00241C70546025463A
:1006D00027469846012000F0B3FBB9F1000F00F067
:1006E0002282994B1B68002B40F01D8217B0BDE899
:1006F000F08F0220FFF778FE002840F00E82944B26
:100700001B88ADF82430022109A800F0B3FAE1E714
:100710004FF47A7000F042FA031E0193EFDB0220DF
:10072000FFF762FE82460028E9D0019B581E04288C
:1007300000F2F581DFE800F0030D1013160016A893
:10074000052340F8343D042100F094FA5446002774
:1007500052E004217848F7E704217E48F4E70421B9
:100760007D48F1E71C24204600F0B8FA04340990D3
:10077000042109A800F07EFA2C2CF4D1E6E7002D24
:10078000BDD0002CBBD00220FFF72EFE054600286E
:1007900000F0C781012000F09FFA022088F80000D5
:1007A00000F04EFB0024E3B21846019300F0A4FAD7
:1007B000824648B1019B184600F0AEFA0134002889
:1007C000F1D12C46654B9BE70123022088F80030CD
:1007D00000F02CFB5646DBF808309E4206D230462D
:1007E00000F07CFA0130ECD10436F4E7564B0026D9
:1007F00088F800605E602C4600F068FB1DB1002C9C
:1008000018BF4FF00009FFF7F7FD63E7002D3FF435
:1008100076AF002C3FF473AF022088F8000000F0A0
:100820000FFB322000F0BAF9B0F1000AC0F2798172
:100830001AF0030540F07581DBF8082006EB0A0387
:10084000934200F26E81BAF5807F00F26A81444BD8
:10085000019355450DDA4FF47A7000F09FF902903C
:10086000029A002AC0F25D81019B029AEA54013586
:10087000EEE7C820FFF7B8FD0546002800F05181DB
:100880001F2E11D8C6F12004544528BF54460EAB84
:1008900026F0030022463249184400F0E5FA2246C9
:1008A000FF212F4800F00AFB4FEAAA0A5FFA8AF2FA
:1008B0002B493046FFF7BEFD0446002881D006EBE9
:1008C0008A06054698E70220FFF78EFD00283FF4D0
:1008D00016AFFFF79FFD00283FF411AF00229246AC
:1008E000DBF808309A4259D21F2A1ED80E9B0133DA
:1008F0001BD022F0030316A90B4453F8203C0993A4
:100900001848436883B3174800210DF1240E11F8ED
:100910000E3083EA0A03DBB2013150F82330042998
:1009200083EA1A2AF3D10432DAE71046019200F082
:10093000D5F9019A0990E3E7502402209C25022072
:100940005C240220CD040008A02902209824022063
:10095000223B00085424022058240220243B000893
:100960009C240220A025022019464FF0080E11F009
:10097000010F4FEA51011FBF81F06D4181F4380131
:1009800081F4034181F02001BEF1010EEFD140F866
:1009900023100133B3F5807FE6D1B4E716A8042114
:1009A00040F84CAD00F066F926E716A8002340F8A1
:1009B000343D642100F02AF900287FF4A0AE022023
:1009C000FFF712FD00283FF49AAE099800F0B6F93F
:1009D00016AB43F8480D04211846E3E716A8002398
:1009E00040F8343D642100F011F900287FF487AE0F
:1009F0000220FFF7F9FC00283FF481AE099800F0CF
:100A0000ABF916AB43F8440DE5E70220FFF7ECFC29
:100A100000283FF474AE00F0A5F916AB43F8400D82
:100A2000D9E70220FFF7E0FC00283FF468AE09A9EF
:100A3000142000F09DF9824616A8042140F83CAD30
:100A400000F018F9514609A8ACE7322000F0A6F8EA
:100A5000B0F1000AFFF653AE1AF0030F7FF44FAE69
:100A6000DBF808200AEB070393423FF648AE02206A
:100A7000FFF7BAFC00283FF442AE2AF0030ABA445A
:100A8000BA453FF4B9AE384600F028F90421089081
:100A900008A800F0EFF80437F2E74FF47A70FFF798
:100AA000A3FC00283FF42BAEFFF7B4FC00283FF472
:100AB00089AE0E9B01330CD008220EA90020FFF74F
:100AC000B9FC00283FF47EAE2022FF210EA800F0E2
:100AD000F5F9FFF791FC304801F088FA06E616A810
:100AE000002340F8343D642100F090F8824600284D
:100AF0007FF405AE0220FFF777FC00283FF4FFAD3E
:100B0000FFF77AFC41F2883001F070FA099800F0A2
:100B100021FAD14600F0DAF9DCE505466CE600275B
:100B2000EDE52546EBE5002000F038F80290029B49
:100B3000002BFFF6D2AD012000F078F9029B213B9B
:100B4000122B3FF6C7AD01A252F823F0F3060008BE
:100B5000110700087F070008D5060008D506000821
:100B6000D50600080D0800084B0A0008C708000851
:100B7000AB090008DD0900080B0A0008D5060008CB
:100B8000230A0008D50600089B0A0008F907000898
:100B9000D5060008DF0A0008A08601002DE9F3470A
:100BA00002AE00244FF47A7506F8014D144FDFF8B9
:100BB0005880454397F900305A1C5FFA84F901D0F8
:100BC000A34212D158F8240003680122D3F820A0D0
:100BD00031462B46D047012807D10A4B9DF8070024
:100BE00083F8009002B0BDE8F0870134022CE1D117
:100BF0004FF4FA7001F0FAF94FF0FF30F2E700BF5E
:100C000000240220C4290220303B00082DE9F047CF
:100C10004FF47A75144FDFF8588006464D43002490
:100C200097F900305A1C5FFA84F901D0A34210D121
:100C300058F8240003680422D3F820A031462B463C
:100C4000D047042805D1094B83F800900020BDE867
:100C5000F0870134022CE3D14FF4FA7001F0C6F9A9
:100C60004FF0FF30BDE8F08700240220C4290220A5
:100C7000303B000830B4074B1A78074B53F822403A
:100C80002368DD69054B0A46AC460146204630BC68
:100C9000604700BFC4290220303B0008A086010045
:100CA000F8B501F0DBFB094C094E0A4F2070002516
:100CB00030682378834207D901F0CAFB33680544C2
:100CC0000133BD423360F3D9F8BD00BFC52902200E
:100CD000A8290220FF7F010001F07EBC00F1006026
:100CE00000F5C0300068704700F10060920000F528
:100CF000C03001F009BC0000054B1A68054B1B7899
:100D00009B1A834202D9104401F0A2BB0020704715
:100D1000A8290220C529022038B5074D04462868B5
:100D2000204401F09DFB28B928682044BDE83840E4
:100D300001F0AEBB38BD00BFA829022010F00303AC
:100D400008D1B0F5806F05D800F10050A0F57120F2
:100D50000068704700207047014BC058704700BFC3
:100D600020F4F01F014B1868704700BF002004E01A
:100D7000F0B5204B1E68204B1F885D6893F9084032
:100D8000C6F30B02BA424FEA164622D09F89BA42F6
:100D900021D01F8BBA4206D102220C2404FB02335D
:100DA0005D6893F90840B6F5805F16D041F2010303
:100DB0009E4208BF5A24421E0A44013D0B469342FC
:100DC00015D215F9016F581C4EB1034600F8016C9D
:100DD000F5E70022E1E70122DFE74124EBE72C25DC
:100DE00082421D7001D9981C5C70401AF0BD1846F3
:100DF000FBE700BF002004E004240220094B5B88CD
:100E0000B3F5805F09D041F20102934207D101227C
:100E1000054B03EB8203D87870470022F8E70020E7
:100E2000704700BF002004E0283B0008022802BFF2
:100E3000024B4FF080629A61704700BF000C024085
:100E4000022802BF024B4FF480629A61704700BFD4
:100E5000000C0240022801BF024A536983F48063F8
:100E600053617047000C024010B50023934203D039
:100E7000CC5CC4540133F9E710BD000030B5441E0A
:100E800014F9010F0B4660B193F90050854201F14E
:100E9000010106D11AB993F90020801A30BD013A38
:100EA000EEE7002AF7D1104630BD000002460346A7
:100EB000981A13F9011B0029FAD17047024403461E
:100EC000934202D003F8011BFAE77047024B1A78ED
:100ED000024B1A70704700BFC42902200024022070
:100EE00038B5164D164C284600F0C0FB2146284662
:100EF00000F0E8FB23681348DA6ED2F8043843F0B8
:100F00000203C2F8043801F071F80F49206800F0BC
:100F1000E7FC23680D48DA6E0D49D2F8043823F057
:100F20000203C2F80438A8424FF4E1330B6003D047
:100F3000BDE8384000F0F8BA38BD00BF742E02207A
:100F4000203C000840420F00743C0008C8290220E1
:100F5000AC29022038B50B4B1A780B4B53F82240C2
:100F60000A4B9C4205460CD0094B0021184618221A
:100F7000FFF7A4FF056001462046BDE8384000F0B9
:100F8000D3BA38BDC4290220303B0008742E022099
:100F9000AC290220024A136843F0C0031360704773
:100FA00000780040044B5A6810439A6858600AB1B0
:100FB000181D1047704700BFC82902202DE9F84FBF
:100FC000404EF56D2F68EC692C62210718D014F0A3
:100FD000080F0CBF00208020E20748BF40F020002F
:100FE000A30748BF40F04000610748BF40F480704D
:100FF000202383F31188FFF7D5FF002383F31188A3
:10100000E20509D5202383F311884FF40070FFF720
:10101000C9FF002383F31188DFF8A8A04FF020094F
:101020004FF0000B14F0200832D13B0615D5DFF845
:1010300098A04FF0200920060FD589F3118850465B
:1010400000F0E6F9002830DA0820FFF7ABFF27F0C0
:1010500080032B60002383F3118879060DD5620687
:101060000BD5202383F31188F26C336D9A4201D1A2
:10107000336CFBB9002383F31188E30604D5B26E09
:1010800013690BB150699847BDE8F84F01F02ABBCE
:1010900089F311886B6A96F864105046194000F085
:1010A00051FA8BF31188EC69BCE7A86288F31188C8
:1010B000EC69C0E7102027F04007FFF773FF2F60AF
:1010C000D8E700BFC8290220002A022013B5104C1F
:1010D000204600F01DFA04F11400009400234FF4A0
:1010E00000720C4900F0DEF804F1380000940A4B5D
:1010F0000A494FF4007200F057F9094BE365094BB8
:1011000023660B21522002B0BDE8104000F058B811
:10111000C8290220342A0220950F0008342C02200E
:101120000078004080F93703224B002908BF194698
:10113000037C8166012B30B50CD11F4B984209D13D
:101140001E4B1A6C42F080421A641A6E42F08042C2
:101150001A661B6E0A68036EC46D03EB5203B3FB81
:10116000F2F34A68150442BF23F0070503F00703B2
:1011700043EA4503E3608B6843F040036360CB6858
:1011800043F00103A36042F4967343F0010323602C
:1011900051054FF0FF33236205D512F0102205D020
:1011A000B2F1805F04D080F8643030BD7F23FAE76D
:1011B0003F23F8E7643B0008C829022000380240BA
:1011C00000F1604300F01F02400903F5614309018B
:1011D0008000C9B200F1604083F8001300F561405F
:1011E00001239340C0F8803103607047F8B515467D
:1011F00082680669AA420B46816938BF8568761AFB
:10120000B542044607D218462A46FFF72DFEA369C9
:101210002B44A3610DE011D932461846FFF724FE96
:10122000AF1B3A46E1683044FFF71EFEE2683A44DD
:10123000A261A3685B1BA3602846F8BD18462A4636
:10124000FFF712FEE368E4E783682DE9F041044606
:1012500093421546266938BF85684069361AB542FB
:101260000F4606D22A46FFF7FFFD63692B446361F0
:101270000DE012D93246A5EB0608FFF7F5FD424610
:10128000B919E068FFF7F0FDE26842446261A368C3
:101290005B1BA3602846BDE8F0812A46FFF7E4FD0A
:1012A000E368E4E710B50A440024C361029B0060D0
:1012B00040608460C160816141610261036210BD70
:1012C00008B582694369934201D1826882B9826814
:1012D000013282605A1C42611970426903699A4264
:1012E00001D3C3684361002100F09CFE002008BDCB
:1012F0004FF0FF3008BD000070B5202304460E46B5
:1013000083F31188A568A5B1A368A269013BA36016
:10131000531CA36115782269934224BFE368A3613B
:10132000E3690BB120469847002383F311882846D0
:1013300070BD3146204600F065FE0028E2DA85F3F4
:10134000118870BD2DE9F74F05460F4690469A4625
:10135000D0F81C90202686F311884FF0000B14461D
:1013600064B1224639462846FFF740FF034668B974
:101370005146284600F046FE0028F1D0002383F3B2
:101380001188A8EB040003B0BDE8F08FB9F1000F9D
:1013900003D001902846C847019B8BF31188E41ABB
:1013A0001F4486F31188DBE7C16081614161C3613D
:1013B0001144009B006040608260016103627047DD
:1013C000F8B504460E461746202383F31188A56816
:1013D000A5B1A368013BA36063695A1C62611E70DA
:1013E000236962699A4224BFE3686361E3690BB1D0
:1013F00020469847002080F31188F8BD39462046E2
:1014000000F000FE0028E2DA85F31188F8BD000044
:10141000836942699A4210B501D182687AB98268BB
:10142000013282605A1C82611C7803699A4201D39E
:10143000C3688361002100F0F5FD204610BD4FF028
:10144000FF3010BD2DE9F74F05460F4690469A46EE
:10145000D0F81C90202686F311884FF0000B14461C
:1014600064B1224639462846FFF7EEFE034668B9C6
:101470005146284600F0C6FD0028F1D0002383F332
:101480001188A8EB040003B0BDE8F08FB9F1000F9C
:1014900003D001902846C847019B8BF31188E41ABA
:1014A0001F4486F31188DBE702684368114301603B
:1014B00003B11847704700001430FFF743BF000026
:1014C0004FF0FF331430FFF73DBF00003830FFF717
:1014D000B9BF00004FF0FF333830FFF7B3BF000053
:1014E0001430FFF709BF00004FF0FF311430FFF751
:1014F00003BF00003830FFF763BF00004FF0FF323A
:101500003830FFF75DBF000000207047FFF7DEBDF9
:10151000044B0360002343608360C36001230374B2
:10152000704700BF7C3B000810B52023044683F3BE
:101530001188FFF7F9FD02232374002383F3118838
:1015400010BD000038B5C36904460D461BB904211F
:101550000844FFF7A9FF294604F11400FFF7B0FE85
:10156000002806DA201D4FF48061BDE83840FFF7FF
:101570009BBF38BD026843681143016003B118473F
:101580007047000013B5446BD4F894341A6811788E
:10159000042915D1217C022912D11979128901233C
:1015A0008B4013420CD101A904F14C0001F0A4FEC0
:1015B000D4F89444019B21790246206800F0E0F9B8
:1015C00002B010BD143001F027BE00004FF0FF3311
:1015D000143001F021BE00004C3001F0F9BE0000D3
:1015E0004FF0FF334C3001F0F3BE0000143001F037
:1015F000F5BD00004FF0FF31143001F0EFBD0000E9
:101600004C3001F0C5BE00004FF0FF324C3001F00D
:10161000BFBE0000D0F8942438B5136819780429A7
:10162000054601D0012038BD017C0229FAD112798A
:101630005C89012090400440F4D105F1140001F0D0
:1016400087FD02460028EDD0D5F894544FF48073FE
:101650002868697900F082F9204638BD406BFFF7B1
:10166000D9BF000000207047704700007FB5124BC3
:101670000360002343608360C360012502260F4B93
:10168000057404460290019300F1840229460096F5
:101690004FF48073143001F037FD094B019302942D
:1016A00000964FF4807304F52372294604F14C0030
:1016B00001F0FEFD04B070BDA43B00085D160008FB
:1016C000851500080B68202282F311880A7903EB44
:1016D000820210624A790D3243F822008A7912B1EF
:1016E00003EB8203186202230374C0F894140023EE
:1016F00083F311887047000038B5037F044613B1A7
:1017000090F85430ABB9201D01250221FFF732FFBC
:1017100004F1140025776FF0010100F08FFC84F8CC
:10172000545004F14C006FF00101BDE8384000F066
:1017300085BC38BD10B5012104460430FFF71AFFFF
:101740000023237784F8543010BD000038B50446D8
:101750000025143001F0F0FC04F14C00257701F075
:10176000BFFD201D84F854500121FFF703FF2046E0
:10177000BDE83840FFF74EBF90F85C3003F06003DF
:10178000202B19D190F85D20212A0AD0222A4FF06F
:1017900000030ED0202A0FD1084A026507224265B5
:1017A00004E0064B0365072343650023836501209E
:1017B000704703654365F9E700207047282402203D
:1017C000D0F8943437B51A681178042904461AD130
:1017D000017C022917D11979128901238B40134208
:1017E00011D100F14C05284601F03AFE58B101A98B
:1017F000284601F081FDD4F89444019B21790246EA
:10180000206800F0BDF803B030BD000000EB81039C
:10181000F7B51C6A05460E46F4B1202383F3118800
:1018200005EB8607201D0821FFF7A4FEFB685B6916
:101830001B684C3413B1204601F06CFD01A9204611
:1018400001F05AFD024648B1019B3146284600F09E
:1018500097F8002383F3118803B0F0BDFB685A6941
:101860001268002AF5D01B8A013B1340F1D105F123
:101870005C02EAE70D3138B550F82140DCB1202395
:1018800083F31188D4F894241368527903EB82030C
:10189000DB689B695D6845B104216018FFF76AFE4B
:1018A000294604F1140001F05DFC2046FFF7B2FE6A
:1018B000002383F3118838BD7047000001F00AB897
:1018C000012303700023436000F1240200F138017A
:1018D00042F8043B8A421361FAD103814381704785
:1018E00038B50446202383F3118800254160C56084
:1018F000056145618561C561056200F0FBFF02235A
:10190000237085F3118838BD70B500EB810305465F
:101910005069DA600E46144618B110220021FFF714
:10192000CDFAA06918B110220021FFF7C7FA31469D
:101930002846BDE8704001F0A7B80000028902F017
:1019400001020281428902F0010242810022026109
:1019500042618261C261026201F02AB9F0B400EB17
:1019600081044789E4680125A4698D403D43458190
:1019700023600023A2606360F0BC01F045B9000061
:10198000F0B400EB81040789E468012564698D40A7
:101990003D43058123600023A2606360F0BC01F039
:1019A000BFB9000070B50223002504460370A0F8FB
:1019B000645080F8665080F8675005814581C560A5
:1019C000056145618561C561056280F84C5000F094
:1019D000F7FF63681B6823B129462046BDE87040C5
:1019E000184770BD436802781B6880F8682005229C
:1019F00002700BB10421184770470000436890F84B
:101A000068201B6802700BB1052118477047000061
:101A100090F84C3070B5044613B1002380F84C3078
:101A200004F15C02204601F0E5F863689B6863BB43
:101A300094F85C5015F0600615D194F85D3005F00F
:101A40007F0545EA032540F202339D4200F00E81F6
:101A50005BD8022D00F0DC803FD8002D00F087809D
:101A6000012D00F0CF800021204601F02FFB002146
:101A7000204601F021FB63681B6813B10621204654
:101A80009847062384F84C3070BD204698470028BC
:101A9000CED094F8632094F8623043EA0223626D5A
:101AA000934238BF636594F95C30656D002B4FF04D
:101AB000200380F2FD80002D00F0EC80092284F8E4
:101AC0004C2083F311880021636D226D2046FFF7BF
:101AD00057FF002383F3118870BDB5F5817F00F0B7
:101AE000B180B5F5407F49D0B5F5807FBBD194F882
:101AF0005E30012BB7D1B4F8643023F00203A4F8B0
:101B0000643026656665A665C3E740F201639D42C1
:101B10001ED8B5F5C06F3BD2B5F5A06FA3D1B4F810
:101B20005C30B3F5A06F0ED194F85E3084F8663067
:101B3000204600F09DFF63681B6813B10121204619
:101B4000984703232370002323656365A365A0E7FB
:101B5000B5F5106F32D040F602439D4252D0B5F534
:101B6000006F80D104F167032365012324E004F1B1
:101B70006403236502236365A5658AE794F85E30F4
:101B8000012B7FF470AFB4F8643043F00203B6E782
:101B900094F86120616894F860304D6894F85F10A3
:101BA00043EA0223204694F85E20A84700283FF429
:101BB0005AAF4368236503686365A4E72378042B61
:101BC00010D1202383F311882046FFF7B7FE86F358
:101BD0001188636884F867601B68032121700BB16A
:101BE0002046984794F85E30002BACD084F86730DC
:101BF0000423237063681B68002BA4D002212046B5
:101C00009847A0E7374B23650223636500239DE7D0
:101C100094F8601011F0800F204601F00F010ED0F3
:101C200000F0DAFF012806D002287FF41CAF2E4B0B
:101C30002365606567E72D4B2365656563E700F005
:101C4000BDFFEFE794F85E30002B7FF40CAF94F803
:101C5000603013F00F013FF476AF1A06204602D52C
:101C600001F048FA6FE701F03BFA6CE794F85E3058
:101C7000002B7FF4F8AE94F8603013F00F013FF4BE
:101C800062AF1B06204602D501F020FA5BE701F0A7
:101C900013FA58E7142284F84C2083F311882B465A
:101CA0002A4629462046FFF759FE85F3118870BD64
:101CB0005DB1152284F84C2083F311880021636DF7
:101CC000226D2046FFF74AFE03E70B2284F84C20E2
:101CD00083F311882B462A4629462046FFF750FEFB
:101CE000E3E700BFD43B0008CC3B0008D03B000832
:101CF00038B590F84C300446152B29D8DFE803F0AE
:101D00003E28282828283E28280B29392828282832
:101D1000282828283E3E90F8631090F86220436DF2
:101D200042EA01229A4214D9C268128AB3FBF2F540
:101D300002FB15356DB9202383F311882B462A4603
:101D40002946FFF71DFE85F311880A2384F84C30DD
:101D500038BD142384F84C30202383F311880023EA
:101D60001A4619462046FFF7F9FD002383F3118830
:101D700038BD836D03B198470023E7E7002101F0E8
:101D8000A5F90021204601F097F963681B6813B19B
:101D90000621204698470623D8E7000090F84C20FB
:101DA000152A38B5044622D80123934040F64162F3
:101DB00013421DD113F480150FD19B0217D50B23AD
:101DC00080F84C30202383F311882B462A4629467D
:101DD000FFF7D6FD85F3118838BDC3689B695B6842
:101DE0002BB9836D03B19847002384F84C3038BD7C
:101DF000002101F06BF90021204601F05DF96368D4
:101E00001B6813B10621204698470623EDE7000022
:101E1000024B00221B605B609A607047342E0220E8
:101E2000002303748268054B1B6899689142FBD2BA
:101E30005A6803604260106058607047342E022078
:101E400008B5202383F31188037C032B05D0042BD2
:101E50000DD02BB983F3118808BD436900221A60A5
:101E60004FF0FF334361FFF7DBFF0023F2E790E819
:101E70000C001A6002685360F2E70000002303744C
:101E80008268054B1B6899689142FBD85A680360C9
:101E90004260106058607047342E0220054B19696B
:101EA0000874186802681A6053601861012303748B
:101EB000FEF73ABA342E022030B54B1C87B00546E7
:101EC0000A4C10D023690A4A01A800F0D3F828462A
:101ED000FFF7E4FF049B13B101A800F007F92369A1
:101EE000586907B030BDFFF7D9FFF8E7342E02205C
:101EF000411E000838B50C4D41612B6981689A6814
:101F00009142044603D8BDE83840FFF789BF184620
:101F1000FFF786FF01232C61014623742046BDE8AC
:101F20003840FEF701BA00BF342E0220044B1A6875
:101F30001B6990689B68984294BF002001207047FD
:101F4000342E022010B5084C236820691A682260DC
:101F50005460012223611A74FFF790FF0146206943
:101F6000BDE81040FEF7E0B9342E02208260022264
:101F700002740022427470478368A3F17C0243F824
:101F80000C2C026943F83C2C426943F8382C074A70
:101F900043F81C2CC26843F8102C022203F8082CCA
:101FA000002203F8072CA3F1180070474103000832
:101FB00010B5202383F31188FFF7DEFF00210446CC
:101FC000FFF798FF002383F31188204610BD00001F
:101FD000024B1B6958610F20FFF760BF342E0220AF
:101FE000202383F31188FFF7F3BF000008B50146F3
:101FF000202383F311880820FFF75EFF002383F37B
:10200000118808BD49B1064B42681B6918605A60C7
:10201000136043600420FFF74FBF4FF0FF3070475D
:10202000342E02200368984206D01A68026050607D
:1020300059611846FFF7F4BE7047000038B50446F2
:102040000D462068844200D138BD036823605C607F
:102050004561FFF7E5FEF4E7054B03F114025A6111
:102060009A614FF0FF32DA6100221A62704700BFB6
:10207000342E0220F8B503614FF08043C2605C6AE1
:10208000194B1A46022952F8145F38BF02219542B3
:1020900006461F460AD1586198611C62056045607A
:1020A00081600819BDE8F84001F0FCB9186AAB6816
:1020B000241A0C1902D3E41A2D6804E09C4202D2BF
:1020C000204401F0FDF9AB689C42F4D86B68736062
:1020D00035601E606E60B460A9684FF0FF33091B65
:1020E000A960FB61F8BD00BF342E022010B41B4C68
:1020F000234653F8141F814210D0416802680A60D9
:10210000026851609A424FF00001C16003D09368A9
:1021100081680B4493605DF8044B70470A68626104
:1021200000209A425360C86003D15DF8044B01F06F
:10213000C1B993688868034493604FF08042206A75
:10214000526A121A9342E6D9991A012998BF931C30
:1021500018445DF8044B01F0B3B900BF342E0220DF
:1021600000207047FEE70000704700004FF0FF308E
:1021700070470000022906D0032906D0012906482D
:1021800018BF0020704705487047032A9ABF0448CB
:1021900000EBC20000207047D03C0008843C0008DF
:1021A0003024022070B5044608460D46FEF77EFE38
:1021B000C6B22046013403780BB9184670BD3246CA
:1021C0002946FEF75BFE0028F3D1012070BD000018
:1021D0002DE9F04F80469BB008460C461646FEF7A8
:1021E00065FE3C49C5B22046FFF7DCFF08B1073564
:1021F000EDB239492046FFF7D5FF08B11035EDB2F1
:10220000632D01AF0CD8DFF8DC90DFF8DCB03D4681
:1022100094F800A0BAF1000F1CD185F800A003E0EB
:102220002146384601F074FC3846FEF73FFEC0B246
:10223000431C5B0088E8480033700323737000235D
:1022400002361946DAB2904206F102063BD81BB0BC
:10225000BDE8F08FBAF1250F30D107221D49204685
:10226000FEF70CFE70B91D4B2A4603F10C0153F822
:10227000040B42F8040B8B42F9D11B8813800734FE
:102280000E35C5E7082214492046FEF7F7FDA8B928
:102290001349AB1C11F8012F100902F00F0210F8BE
:1022A000090012F8092003F8020C594503F8012C23
:1022B00003F10203EED118350834A9E785F800A030
:1022C00001340135A4E7FA5C06F8022C06F8011C7B
:1022D0000133B7E7283C0008303C0008393C0008CF
:1022E0001FF4F01F483C00082BF4F01F08B5202312
:1022F00083F311880348FFF763FA002383F31188FF
:1023000008BD00BF742E022010B50446052916D85A
:10231000DFE801F016150316161D202383F311883C
:102320000E4A0121FFF7F0FA20460D4A0221FFF77D
:10233000EBFA0C48FFF70AFA002383F3118810BD6B
:10234000202383F311880748FFF7D6F9F4E7202309
:1023500083F311880348FFF7EDF9EDE7D83B000858
:10236000FC3B0008742E022038B50C4D0C4C0D4976
:102370002A4604F10800FFF72BFF05F1CA0204F119
:1023800010000949FFF724FF05F5CA7204F118008F
:102390000649BDE83840FFF71BBF00BF3C330220B1
:1023A000302402205C3C0008663C0008303C0008F9
:1023B000BFF34F8F024AD368DB03FCD4704700BFE2
:1023C000003C024008B5074B1B7853B9FFF7F0FFFC
:1023D000054B1A69002ABFBF044A5A6002F18832CD
:1023E0005A6008BD9A350220003C0240230167452F
:1023F00008B5054B1B7833B9FFF7DAFF034A1369B9
:1024000043F00043136108BD9A350220003C0240AE
:102410000B2870B513D80B4A0B4C137863B90B4ECD
:102420004FF0006144F8231056F8235001330C2B71
:102430002944F7D10123137054F8200070BD002007
:1024400070BD00BFCC3502209C350220F03C000856
:10245000014B53F820007047F03C00080C207047F7
:102460000B2810B5044601D9002010BDFFF7D0FF9E
:10247000064B53F824301844C21A0BB9012010BD82
:1024800012680132F0D1043BF6E700BFF03C0008CF
:102490000B2810B504462FD8FFF78AFFFFF792FFED
:1024A0001649F323CB60FFF783FFC300DBB243F48D
:1024B000007343F002030B610B6943F480330B613B
:1024C000FFF776FFFFF7A4FF0D4B53F824300344CA
:1024D000BFF34F8F0B4A98420AD3BFF34F8FBFF31E
:1024E0006F8FFFF785FF2046BDE81040FFF7B8BFAC
:1024F000C2F85C022030EEE7002010BD003C024034
:10250000F03C000800ED00E02DE9F84312F0010373
:10251000154643D10244B2F1026F3FD22C4B1B68E7
:1025200013F001033AD02B4CFFF74CFFF323E36089
:10253000FFF73EFF40F20127032D16D8254C0F462A
:10254000401A40F20118EB1B0B44012B00EB07066D
:10255000236926D823F001032361FFF749FF0120F7
:10256000BDE8F883043D0430E6E78307E6D123693C
:1025700023F44073236123693B43236151F8046BC7
:102580000660BFF34F8FFFF713FF03689E42E9D049
:10259000236923F001032361FFF72AFF0020BDE830
:1025A000F88323F440732361236943EA080323611A
:1025B000B94637F8023B3380BFF34F8FFFF7F8FE81
:1025C0003688B9F80030B6B2B342BCD0E0E700BFFD
:1025D00000380240003C0240084908B50B7828B199
:1025E00053B9FFF7EFFE01230B7008BD23B1BDE81F
:1025F00008400870FFF7FCBE08BD00BF9A350220F6
:1026000010B50244064B0439D2B2904200D110BD3D
:10261000441C00B253F8200041F8040FE0B2F4E784
:1026200050280040104B30B51C6F240407D41C6F99
:1026300044F400741C671C6F44F400441C670B4C8A
:10264000236843F4807323600244094B0439D2B2F7
:10265000904200D130BD441C00B251F8045F43F8F1
:102660002050E0B2F4E700BF0038024000700040A4
:102670005028004007B5012201A90020FFF7C0FF44
:10268000019803B05DF804FB07B502A9012241F8E7
:10269000040D0020FFF7C6FF03B05DF804FB000047
:1026A000034B1B689B0042BF024B01221A7070470C
:1026B00074380240CD350220014B1878704700BFB6
:1026C000CD350220064A536823F001035360EFF32F
:1026D0000983683383F30988002383F311887047E3
:1026E00030EF00E010B5202383F31188104B5B68B6
:1026F00013F4006318D0F1EE103AEFF309844FF0B1
:10270000807344F84C3C0B4BDB6844F8083CA4F164
:10271000680383F30988FFF709FC18B1064B44F8F6
:10272000503C10BD054BFAE783F3118810BD00BF84
:1027300000ED00E030EF00E0510300085403000812
:10274000F0B5BFF34F8FBFF36F8F1D4B0021C3F860
:102750005012BFF34F8FBFF36F8F5A6942F40032AC
:102760005A61BFF34F8FBFF36F8FC3F88410BFF36D
:102770004F8FD3F88020C2F3C904C2F34E32520106
:10278000A50743F6E07602EA060E284621464EEA01
:1027900000070139C3F860724F1C00F14040F6D1C8
:1027A000203A12F1200FEED1BFF34F8F5A6942F455
:1027B00080325A61BFF34F8FBFF36F8FF0BD00BF00
:1027C00000ED00E0FEE70000084A094B09498B4292
:1027D00004D3094A0021934205D3704752F8040FED
:1027E00043F8040BF3E743F8041BF4E7FC3E00084E
:1027F000D8380220D8380220D8380220036F30B5EC
:1028000000229D68C46E11464FF0FF3004EB421366
:1028100001329542C3F80019C3F81019C3F808092A
:10282000C3F8001BC3F8101BC3F8080BEED24FF01F
:102830000113C4F81C3830BD890141F02001016149
:1028400003699B06FCD4122000F0C8BE204B03EBAA
:1028500080022DE9F047D2F80CE0DD6EDEF814209E
:10286000461CD2F800C005EB063605EB401851684F
:1028700061450BD3D5F83428012303FA00F022EA8E
:102880000000C5F834081846BDE8F087BEF81040CF
:10289000ACEB0103A34228BF2346D8F81849A4B2E1
:1028A000B3EB840F10D894681F46A4F1040959F8BB
:1028B00004AFC6F800A0042F01D9043FF7E71C4479
:1028C0000B4494605360D2E70020BDE8F08700BF5E
:1028D000D035022010B5054C2046FEF7F1FF4FF031
:1028E000A043E366024B236710BD00BFD035022032
:1028F000443D00080378012B70B5054650D12A4BA2
:10290000C46E98421BD1294B5A6B42F080025A6325
:102910005A6D42F080025A655A6D5A6942F080023F
:102920005A615A6922F080025A610E2143205B6984
:10293000FEF746FC1E4BE3601E4BC4F80038002334
:10294000C4F8003EC0232360EE6E4FF40413A3636B
:102950003369002BFCDA012333610C2000F03EFECA
:102960003369DB07FCD4122000F038FE3369002BFA
:10297000FCDA0026A6602846FFF740FF6B68C4F823
:102980001068DB68C4F81468C4F81C684BB90A4BBB
:10299000A3614FF0FF336361A36843F00103A360B9
:1029A00070BD064BF4E700BFD0350220003802406E
:1029B0004014004003002002003C30C0083C30C0FE
:1029C000F8B5C46E054600212046FFF735FF296F94
:1029D00000234FF001128F68C4F834384FF00066BE
:1029E000C4F81C284FF0FF3004EB431201339F4220
:1029F000C2F80069C2F8006BC2F80809C2F8080BF7
:102A0000F2D20B68EA6E6B6763621023136116697A
:102A100016F01006FBD1122000F0E0FDD4F80038CB
:102A200023F4FE63C4F80038A36943F4402343F061
:102A30001003A3610923C4F81038C4F814380A4BF2
:102A4000EB604FF0C043C4F8103B084BC4F8003BA8
:102A5000C4F81069C4F800396B6F03F1100243F435
:102A600080136A67A362F8BD203D00084080001013
:102A7000C26E90F86610D2F8003823F4FE6343EA81
:102A80000113C2F8003870472DE9F0410EB200EB97
:102A900086080D46D8F80C100F6807F00303022BC8
:102AA00050D0032B50D03D4A3D4F012B18BF174645
:102AB000C46E4FEA451E04EB0E030022C3F8102B30
:102AC0008A6905F1100C002A40D04A8A05F15803A2
:102AD0005B013A43E2500123D4F81C2803FA0CF3BB
:102AE0001343A6444A69C4F81C380023CEF81039B1
:102AF00005F13F03002A39D00A8A898B92080129FF
:102B000088BF4A43416F04EB8303561841EA0242EF
:102B1000466729465A602046FFF78EFED8F80C30EB
:102B20001B8A43EA85531F4305F148035B01E750C5
:102B30000123D4F81C2803FA05F51543C4F81C58E2
:102B4000BDE8F081174FB3E7174FB1E704EB461329
:102B5000D3F8002B22F40042C3F8002BD4F81C2831
:102B6000012303FA0CF322EA0303BAE704EB83031D
:102B70000E4A5A6004EB461629462046FFF75CFED3
:102B8000D6F8003923F40043C6F80039D4F81C38CD
:102B9000012202FA05F523EA0505CFE700800010BF
:102BA000008004100080081000800C100004000257
:102BB000026F12684267FFF721BE00005831C36EF2
:102BC00049015B5813F4004004D013F4001F14BFF4
:102BD00001200220704700004831C36E49015B5854
:102BE00013F4004004D013F4001F14BF012002208E
:102BF0007047000000EB8101CB68196A0B68136015
:102C00004B6853607047000000EB810330B5DD680E
:102C1000AA691368D36019B9402B84BF402313609D
:102C20006B8A1468C26E1C44013CB4FBF3F463432A
:102C3000033323F0030302EB411043EAC44343F0A0
:102C4000C043C0F8103B2B6803F00303012B09B20B
:102C50000ED1D2F8083802EB411013F4807FD0F87F
:102C6000003B14BF43F0805343F00053C0F8003BD7
:102C700002EB4112D2F8003B43F00443C2F8003BA0
:102C800030BD00002DE9F041244DEE6E06EB4013FF
:102C90000446D3F8087BC3F8087B38070AD5D6F872
:102CA0001438190706D505EB84032146DB6828464E
:102CB0005B689847FA072FD5D6F81438DB072BD571
:102CC00005EB8403D968CCB98B69488A5E68B6FB8A
:102CD000F0F200FB12628AB91868DA6890420DD2ED
:102CE000121A83E81400202383F311880B4821462D
:102CF000FFF78AFF84F31188BDE8F081012303FA0E
:102D000004F26B8923EA02036B81CB6823B121466D
:102D10000248BDE8F0411847BDE8F081D0350220F7
:102D200000EB810370B5DD68C36E6C692668E660F0
:102D30004A0156BB1A444FF40020C2F810092A6811
:102D400002F00302012A0AB20ED1D3F8080803EBFD
:102D5000421410F4807FD4F8000914BF40F0805072
:102D600040F00050C4F8000903EB4212D2F8000909
:102D700040F00440C2F80009D3F83408012202FAF6
:102D800001F10143C3F8341870BD19B9402E84BF56
:102D90004020206020682E8A841940F00050013CB9
:102DA0001A44B4FBF6F440EAC440C6E7F8B504465A
:102DB0001E48C56E05EB4413D3F80869C3F80869CB
:102DC000F10717D5D5F81038DA0713D500EB8403CF
:102DD000D9684B691F68DA68974218D2D21B00275E
:102DE0001A605F60202383F311882146FFF798FF64
:102DF00087F31188330617D5D5F834280123A3406B
:102E0000134211D02046BDE8F840FFF71FBD012353
:102E100003FA04F2038923EA020303818B68002B7F
:102E2000E8D021469847E5E7F8BD00BFD03502203D
:102E3000A0482DE9F84FC56E6E69AB691E4016F4C7
:102E4000805F6E61044605D0FEF7ACFDBDE8F84F2B
:102E5000FFF748BC002E12DAD5F8003E95489B07D4
:102E60001EBFD5F8003E23F00303C5F8003ED5F899
:102E7000043823F00103C5F80438FEF7BFFD370519
:102E800002D58C48FEF7AEFDB0040CD5D5F8083855
:102E900013F0060FEB6823F470530CBF43F4105388
:102EA00043F4A053EB60310704D56368DB680BB1D2
:102EB00080489847F2026FD4B3020CD5D4F86C80E6
:102EC000DFF8F0A100274FF00109236F9B68F9B2EA
:102ED0008B4280F09C80F70619D5E16E0A6AC2F336
:102EE0000A1702F00F0302F4F012B2F5802F00F07F
:102EF000B680B2F5402F0AD104EB830301F580516F
:102F0000DB68186A00231A469F4240F09C80330316
:102F1000D5F818481DD5E70302D50020FFF7B2FE0B
:102F2000A50302D50120FFF7ADFE600302D5022004
:102F3000FFF7A8FE210302D50320FFF7A3FEE2025C
:102F400002D50420FFF79EFEA30202D50520FFF75D
:102F500099FE77037FF57AAFE60702D50020FFF7E9
:102F600025FFA50702D50120FFF720FF600702D546
:102F70000220FFF71BFF210702D50320FFF716FFF2
:102F8000E20602D50420FFF711FFA3067FF55EAF2E
:102F90000520FFF70BFF59E7D4F86C80DFF814A188
:102FA00000274FF00109236F9B685FFA87FB5B45A1
:102FB00082D308EB4B13D3F8002902F44022B2F578
:102FC000802F22D1D3F80029002A1EDAD3F8002955
:102FD00042F09042C3F80029D3F80029002AFBDB15
:102FE0005946E06EFFF728FC228909FA0BF322EA22
:102FF0000303238104EB8B03DB689B6813B1594601
:10300000504698475846FFF721FC0137CBE708EBBD
:103010004112D2F8003B03F44023B3F5802F10D1C6
:10302000D2F8003B002B0CDA628909FA01F322EA9C
:103030000303638104EB8103DB68DB680BB150465B
:103040009847013741E79C0708BF0A68072B98BFDC
:10305000027003F101039CBF120A013054E70233EE
:1030600004EB830201F58051526890690268D0F840
:1030700008C04068A2EB000E0022104697420AD119
:1030800004EB830463689B699A683A449A605A68BF
:1030900017445F603BE712F0030F08BF08689645CE
:1030A00088BF8CF8000002F1010284BF000A0CF115
:1030B000010CE3E7D0350220C36E03EB4111D1F8D8
:1030C000003B43F40013C1F8003B7047C36E03EBB1
:1030D0004111D1F8003943F40013C1F800397047A9
:1030E000C36E03EB4111D1F8003B23F40013C1F888
:1030F000003B7047C36E03EB4111D1F8003923F454
:103100000013C1F80039704730B5039C01720433D5
:1031100004FB0325C361049B03630021059B00603E
:103120004060C16042610261856104624262816205
:10313000C162436330BD00000022416A4161016108
:10314000C2608262C2626FF00101FEF777BF0000C9
:1031500003694269934203D1C2680AB100207047F3
:10316000181D704703691960C2680132C260C269E4
:10317000134482690361934224BF436A03610021BF
:10318000FEF750BF38B504460D46E3683BB16269AF
:10319000131D1268A3621344E362002038BD237A32
:1031A00033B929462046FEF72DFF0028EDDA38BD59
:1031B0006FF00100FBE70000C368C269013BC36018
:1031C0004369134482694361934224BF436A436164
:1031D00000238362036B03B11847704770B5202347
:1031E000044683F31188866A3EB9FFF7CBFF054694
:1031F00018B186F31188284670BDA36AE26A13F8F5
:10320000015BA362934202D32046FFF7D5FF002360
:1032100083F31188EFE700002DE9F84F04460E46CE
:1032200090469946202787F311880025AA46D4F8AE
:1032300028B0BBF1000F09D149462046FFF7A2FF95
:1032400020B18BF311882846BDE8F88FA16AE36AA4
:10325000A8EB050B5B1A9B4528BF9B46BBF1400FB3
:103260001BD9334601F1400251F8040B43F8040B1B
:103270009142F9D1A36A40334036A3624035A26A35
:10328000E36A9A4202D32046FFF796FF8AF3118839
:103290004545D8D287F31188C9E730465A46FDF72D
:1032A000E3FDA36A5B445E44A3625D44E7E700007C
:1032B00010B5029C0172043303FB0421C361002397
:1032C0008362C362039B0363049B00604060C4602D
:1032D00042610261816104624262436310BD000089
:1032E000026AC260426A4261026100228262C26274
:1032F0006FF00101FEF7A2BE436902699A4203D151
:10330000C2680AB100207047184650F8043B0B60B1
:1033100070470000C368C2690133C3604369134446
:1033200082694361934224BF436A43610021FEF7EF
:1033300079BE000038B504460D46E3683BB1236909
:103340001A1DA262E2691344E362002038BD237AA9
:1033500033B929462046FEF755FE0028EDDA38BD80
:103360006FF00100FBE7000003691960C268013AD1
:10337000C260C269134482690361934224BF436AF5
:10338000036100238362036B03B118477047000099
:1033900070B5202304460E4683F31188856A35B93B
:1033A0001146FFF7C7FF10B185F3118870BDA36AFE
:1033B0001E70A36AE26A01339342A36204D3E169F7
:1033C00020460439FFF7D0FF002080F3118870BD3C
:1033D0002DE9F84F04460D4691469A464FF02008D5
:1033E00088F311880026B346A76A4FB95146204694
:1033F000FFF7A0FF20B187F311883046BDE8F88FB2
:10340000A06AE76AA9EB06033F1A9F4228BF1F463E
:10341000402F1BD905F1400355F8042B40F8042B2D
:103420009D42F9D1A36A4033A3624036A26AE36A9F
:103430009A4204D3E16920460439FFF795FF8BF3E4
:1034400011884E45D9D288F31188CDE729463A46EE
:10345000FDF70AFDA36A3B443D44A3623E44E5E711
:10346000026943699A4203D1C3681BB91846704781
:103470000023FBE7836A002BF8D0043B9B1AF5D0AE
:103480001360C368013BC360C3691A448369026166
:103490009A4224BF436A0361002383620123E5E764
:1034A00000F042B94FF08043002258631A610222B3
:1034B000DA6070474FF080430022DA607047000006
:1034C0004FF0804358637047FEE7000010B5194C79
:1034D000FEF79EFCFEF7C0FD802217492046FEF74E
:1034E00045FD012344F8180C0374144B144AD968A1
:1034F00021F4E0610904090C0A431249DA60CA6840
:1035000042F08072CA60104A1049C2F8B01F1168B8
:1035100041F0010111601022DA77202283F8222085
:10352000002383F3118862B60948BDE81040FEF716
:103530003FBD00BF5C2E0220503D000800ED00E0C2
:103540000003FA05F0ED00E0001000E055CEACC538
:10355000583D00082DE9F84F1F4C4FF000086569F1
:1035600004F11407C1464FF08043266A5B6AAA68DB
:103570009E1B96421DD34FF0200AAA68236AD5F8F5
:103580000CB0134423622B68BB425F60A6EB0206BB
:103590006361C5F80C8001D1FFF78CFF89F31188B6
:1035A0002869D8478AF311886569AB689E42E4D2DE
:1035B000D9E76269BA420CD0916823628E1B96608B
:1035C000A86802282CBF1818981CBDE8F84FFFF710
:1035D00077BFBDE8F88F00BF342E0220034B596837
:1035E0005A68521A9042FBD8704700BF001000E0A2
:1035F0004B6843608B688360CB68C3600B69436131
:103600004B6903628B6943620B680360704700007B
:1036100008B5274B27481A6940F2FF710A431A611F
:103620001A6922F4FF6222F007021A611A691A6B02
:103630000A431A631A6D0A431A651F4A1B6D114625
:10364000FFF7D6FF1D4802F11C01FFF7D1FF1C4810
:1036500002F13801FFF7CCFF1A4802F15401FFF7DD
:10366000C7FF194802F17001FFF7C2FF174802F1C6
:103670008C01FFF7BDFF164802F1A801FFF7B8FF64
:10368000144802F1C401FFF7B3FF134802F1E0014F
:10369000FFF7AEFF114802F1FC01FFF7A9FF104848
:1036A00002F58C71FFF7A4FFBDE8084000F09EB85A
:1036B0000038024000000240783D0008000402404B
:1036C00000080240000C02400010024000140240BA
:1036D00000180240001C024000200240002402406A
:1036E0000028024008B500F0F5F9FFF7EFFEFEF7FD
:1036F000D7FFBDE80840FEF737BE00007047000066
:103700004FF0804310B51A69920708D500241C6158
:10371000202383F31188FFF71DFF84F31188BDE890
:103720001040FEF7DFBF0000104B1A6C42F00102A0
:103730001A641A6E42F001021A660D4A1B6E9368F3
:1037400043F0010393604FF080436B229A624FF085
:10375000FF32DA6200229A615A63DA605A6001220B
:103760005A6108211A601C20FDF72ABD003802406A
:10377000002004E01B4B1A696FEA42526FEA525272
:103780001A611A69C2F30A021A614FF0FF301A690E
:103790005A69586100215A6959615A691A6A62F076
:1037A00080521A621A6A02F080521A621A6A5A6ABF
:1037B00058625A6A59625A6A0B4A106840F480701B
:1037C0001060186F00F44070B0F5007F1EBF4FF41A
:1037D000803018671967536823F40073536000F052
:1037E00059B900BF0038024000700040354B364ADE
:1037F0001A64364A4FF4404111601A6842F00102DF
:103800001A601A689207FCD59A6822F003029A603F
:103810002C4B19469A6812F00C02FBD1186800F084
:10382000F90018609A601A6842F480321A600B68D6
:103830009B03FCD54B6F43F001034B67214B5A6F41
:103840009007FCD5224A5A601A6842F080721A60CA
:103850001E4B1A4659684904FCD5196841F4803159
:1038600019605368D803FCD5136843F40033136020
:10387000164A53689903FCD5124B1A689201FCD57D
:10388000144A9A6040F20112C3F88C200022C3F857
:103890009020114A40F2073111609A6842F002020A
:1038A0009A60084B9A6802F00C02082AFAD15A6C06
:1038B00042F480425A645A6E42F480425A665B6E09
:1038C000704700BF00380240000400100070004044
:1038D000086C400900948838003C0240084A08B54A
:1038E000536911680B4003F00103536123B1054A8A
:1038F00013680BB150689847BDE80840FEF7F2BE68
:10390000003C014058380220084A08B55369116844
:103910000B4003F00203536123B1054A93680BB1D6
:10392000D0689847BDE80840FEF7DCBE003C014087
:1039300058380220084A08B5536911680B4003F053
:103940000403536123B1054A13690BB150699847C9
:10395000BDE80840FEF7C6BE003C014058380220D2
:10396000084A08B5536911680B4003F00803536116
:1039700023B1054A93690BB1D0699847BDE8084067
:10398000FEF7B0BE003C014058380220084A08B596
:10399000536911680B4003F01003536123B1054ACA
:1039A000136A0BB1506A9847BDE80840FEF79ABE0B
:1039B000003C014058380220174B10B55C691A686A
:1039C000144004F478725A61A30604D5134A936A2A
:1039D0000BB1D06A9847600604D5104A136B0BB13F
:1039E000506B9847210604D50C4A936B0BB1D06BF2
:1039F0009847E20504D5094A136C0BB1506C9847FF
:103A0000A30504D5054A936C0BB1D06C9847BDE86B
:103A10001040FEF767BE00BF003C0140583802204E
:103A20001A4B10B55C691A68144004F47C425A6160
:103A3000620504D5164A136D0BB1506D98472305E6
:103A400004D5134A936D0BB1D06D9847E00404D5AB
:103A50000F4A136E0BB1506E9847A10404D50C4A5F
:103A6000936E0BB1D06E9847620404D5084A136F69
:103A70000BB1506F9847230404D5054A936F0BB1DF
:103A8000D06F9847BDE81040FEF72CBE003C0140C7
:103A900058380220062108B50846FDF791FB06219B
:103AA0000720FDF78DFB06210820FDF789FB062185
:103AB0000920FDF785FB06210A20FDF781FB062181
:103AC0001720FDF77DFB06212820BDE80840FDF703
:103AD00077BB000008B5FFF74DFE00F00DF8FDF7CD
:103AE00015FDFDF7EBFEFDF7BFFDFFF707FEBDE897
:103AF0000840FFF7D5BC0000002304491A465A507D
:103B0000C8180833802B4260F9D17047583802201A
:103B1000034611F8012B03F8012B002AF9D1704755
:103B200012101213121100000010410001105A006F
:103B3000742E0220C829022053544D3332463F3F91
:103B40003F3F3F3F0053544D333246375B347C3563
:103B50005D780053544D333246375B367C375D78A1
:103B600000000000009600000000000000000000BF
:103B70000000000000000000000000000000000045
:103B8000D5140008C1140008FD140008E914000849
:103B9000F5140008E1140008CD140008B914000859
:103BA0000915000800000000E1150008CD15000807
:103BB00009160008F515000801160008ED150008A3
:103BC000D9150008C515000865160008000000009A
:103BD00001000000000000000200000000000000E2
:103BE0000D18000875180008400040000C33022032
:103BF0001C3302200200000000000000030000004F
:103C000000000000B91800080000000010000000CB
:103C10002C33022000000000010000000000000022
:103C2000D03502200101020025424F4152442500B7
:103C30002553455249414C25004D6174656B46370B
:103C400036352D57696E67003031323334353637AB
:103C500038394142434445460000000041726475D2
:103C600050696C6F740025424F415244252D424CDF
:103C700000000000092300087521000879170008DA
:103C8000ED220008430000008C3C000809024300BC
:103C9000020100C0320904000001020201000524F3
:103CA000001001052401000104240202052406007D
:103CB00001070582030800FF09040100020A000051
:103CC00000070501024000000705810240000000D6
:103CD00012000000D83C0008120110010200004050
:103CE0008304405700020102030100000403090499
:103CF00000800000008000000080000000800000C4
:103D000000000200000004000000040000000400A5
:103D10000000040000000400000004000000040093
:103D200000000000111A0008F11C00089D1D000889
:103D300040004000483602204836022001000000C2
:103D400058360220800000004001000005000000FD
:103D50006D61696E00000000703D00086036022051
:103D60005838022001000000C9340008000000009B
:103D700069646C65000000000000802A00000000FB
:103D8000AAAAAAAA00000000FFFF0000000000008D
:103D900000A00A000000000000000000AAAAAAAAD1
:103DA00000000000FFFF0000000000000000000015
:103DB0000000000000000000AAAAAAAA000000005B
:103DC000FFFF0000000000000000000000001000E5
:103DD00000000000AAAAAAAA00000000FFFB000041
:103DE0000000000000000000008002000000000051
:103DF000AAAAAAAA00400100FFFF0000000000805C
:103E0000080000000000000000000000AAAAAAAA02
:103E100000000000FFFF00000000000000000000A4
:103E20000000000000000000AAAAAAAA00000000EA
:103E3000FFFF000000000000000000000000000084
:103E400000000000AAAAAAAA00000000FFFF0000CC
:103E50000000000000000000000000000000000062
:103E6000AAAAAAAA00000000FFFF000000000000AC
:103E70000000000000000000000000000000000042
:103E80000000000000000000000000000000000032
:103E90000000000000000000000000000000000022
:103EA0000000000000000000000000000000000012
:103EB000FF00000000000000383B00083F00000049
:103EC00049040000453B00083F0000005104000089
:103ED000533B00083F00000000960000000008006F
:103EE00004000000EC3C000800000000000000009E
:103EF00000000000000000000000000000000000C2
:00000001FF
